:10000000830100308A00042820308400213017202A
:100010002130840047301720A0308400D2301720D0
:1000200083010A128A11342904068001840A040615
:1000300003190034142883120313C700C81B29288E
:10004000481B312848088A004708C70A0319C80A0C
:1000500082008313481883174708C70A84000008E2
:1000600008008301480C1F39831203178F00031304
:10007000470C03178D0083168C170C14000000002A
:1000800083120C08830147184B28831203178C1B1B
:1000900003140E0D83017F3908007410ED326538AA
:1000A0006139753A65396910A039E4126410E73294
:1000B0006539F3326310EC32E939F33A6800EC3217
:1000C0006F3677106134273AA0396537A03B6F321D
:0C00D0008031653AF036A51E20328021F8
:1000DE003230A100A10B7128031383120800831282
:1000EE000313A600C7309F05261C7E287F28802874
:1000FE009F1583120313A61C8528862887281F1692
:10010E0083120313261D8C288D288E289F160A1203
:10011E008A116F200A128A111F1595288312031354
:10012E001F199A289D281F189E289D28A0289F28B1
:10013E009528831203131E08A428031383120800A4
:10014E00831603131114AB28831603131118B0284A
:10015E00B128AB28831603139112111783128C1139
:10016E00C4309300BA28831203138C1DBF28C028F5
:10017E00BA28831203138C118316111BC728CA28A1
:10018E0083128615CC28831286118316031311173A
:10019E0083128C119301D328831203138C1DD8283C
:1001AE00D928D328831203138C118316111BE02830
:1001BE00E32883128615E52883128611831603130E
:1001CE0011179114EA28831603139118EF28F028BB
:1001DE00EA2883160313911283128C11C5309300F3
:1001EE00F828831203138C1DFD28FE28F82883128D
:1001FE0003138C1183169115042983160313141CF3
:10020E0009290A290429831203131308A200213095
:10021E00A3001229122983120313A30B17291829DD
:10022E0011298316031311161C2983160313111A91
:10023E00212922291C298316031311152629831619
:10024E00031311192B292C29262983120313861522
:10025E00220831290313831208000A128A15732407
:10026E000A128A110A128A15F0240A128A110A1227
:10027E008A154C240A128A110A128A1527240A1288
:10028E008A110A128A154A250A128A11A3004030D1
:10029E000A128A153E240A128A11D230A700403063
:1002AE00A8002308F000F101F01BF1037008A40070
:1002BE007108A5002430A6000A128A114C250A12D4
:1002CE008A1106186B296C29802920186F2970292C
:1002DE007F290530A6000330A700BD30A8004030AE
:1002EE00A90000300A128A11CE210A128A11201496
:1002FE00832983120313201083120313051A8829EE
:10030E008929C729A0188C298D29C62900300A12DF
:10031E008A1176200A128A11A20000300A128A155A
:10032E003E240A128A11D230A7004030A8002208BB
:10033E00A400A5012430A6000A128A114C250A1227
:10034E008A119A30A7004030A8002208A400A50107
:10035E002430A600A0300A128A1140230A128A11F4
:10036E000530A6000330A700A030A8008030A900F9
:10037E0000300A128A11CE210A128A11A014CA293B
:10038E0083120313A01048290A128A11042883121B
:10039E000313AA018611831611148312AB00D729F9
:1003AE00831603131118DC29DD29D72983160313AD
:1003BE009112111783128C11C4309300E629831207
:1003CE0003138C1DEB29EC29E629831203138C11E0
:1003DE008316111BF329F62983128615F829831229
:1003EE00861183160313111783128C119301FF29A3
:0203FE00831268
:1004000003138C1D042A052AFF29831203138C1160
:100410008316111B0C2A0F2A83128615112A8312A8
:10042000861183160313111783128C119301182A56
:10043000831203138C1D1D2A1E2A182A83120313EC
:100440008C118316111B252A282A831286152A2A25
:100450008312861183160313111783128C112B0834
:100460009300322A831203138C1D372A382A322A2A
:10047000831203138C118316111B3F2A422A831205
:100480008615442A831286118316031311178312CB
:100490008C11260893004C2A831203138C1D512AB9
:1004A000522A4C2A831203138C118316111B592ACA
:1004B0005C2A831286155E2A831286118316031323
:1004C000111783128C1127089300662A83120313D5
:1004D0008C1D6B2A6C2A662A831203138C118316D7
:1004E000111B732A762A83128615782A83128611A5
:1004F000831603131117A42A831203138C112A08DD
:100500002807C7002908C80047080318C80A0A12A4
:100510008A111B200A128A119300AA0A8F2A8312B9
:1005200003138C1D942A952A8F2A831203138C118E
:100530008316111B9C2A9F2A83128615A12A8312D7
:100540008611831603131117831203132A08280731
:10055000C7002908C80047080318C80A0A128A11E8
:100560001B200A128A110038031DB72AB82A7C2AD8
:10057000831203138C119301BD2A831203138C1D64
:10058000C22AC32ABD2A831203138C118316111B9E
:10059000CA2ACD2A83128615CF2A83128611831682
:1005A000031311171115D42A831603131119D92A0D
:1005B000DA2AD42A831603131114DE2A83160313AE
:1005C0001118E32AE42ADE2A831603139112111765
:1005D00083128C11C4309300ED2A831203138C1DF7
:1005E000F22AF32AED2A831203138C118316111BAE
:1005F000FA2AFD2A83128615FF2A83128611831692
:100600000313111783128C119301062B831203130A
:100610008C1D0B2B0C2B062B831203138C118316B2
:10062000111B132B162B83128615182B8312861180
:1006300083160313111783128C1140309300202B63
:10064000831203138C1D252B262B202B83120313BF
:100650008C118316111B2D2B302B83128615322BF8
:10066000831286118316031311171115372B831666
:10067000031311193C2B3D2B372B03138312080056
:1006800083120313AF00AD012608AA00342D2E08F3
:10069000253A031D252DFF30AB00AC01A901E72C45
:1006A000AF080319572B2F088400831380012D08EE
:1006B00008000230AA072A02840083130008232DB1
:1006C000A90A662B0830AB07FE30AB070230AA0739
:1006D0002A02840083130008B000840A0008B100D5
:1006E0002918B11F7A2BB009B109B00A0319B10A50
:1006F000AC037B2BA9010B30AB072B08F200F301F5
:100700003108F1003008F0000A128A11C62770087B
:10071000AE002B08F200F3013008F0003108F100C0
:100720000A128A11C6270A128A117408B0007508C5
:10073000B100B201B20AB30133083102031DA22B8A
:1007400032083002031CC72B2B08F200F3013208D9
:10075000F0003308F1000A128A155E240A128A1189
:100760007408B2007508B300AC039C2BAD0AAF0847
:100770000319C12B2F088400831320308000AF0A97
:10078000C72B20300A128A1525240A128A11AC03BD
:100790002C08803A7F3E0318B62B291CDE2BAD0AAD
:1007A000AF080319DA2B2F08840083132D30800043
:1007B000AF0ADE2B2D300A128A1525242B08F200F1
:1007C000F3013208F0003308F1000A128A11C6273B
:1007D0000A128A117408B2007508B30032040319B2
:1007E0001D2C3308F3003208F2003108F100300804
:1007F000F0000A128A11C6277408F0007508F1008B
:100800002B08F200F3010A128A11C6270A128A1174
:100810007008AC00803A763E031C102C0730AC0701
:10082000AD0AAF0803191A2C2F08840083132C0873
:10083000303ED72B2C08303EDB2B0A302E02031C17
:10084000232C0730AE07AD0AAF0803192D2C2F0853
:10085000840083132E08303E2D2D2E08303E312D7E
:10086000AD0AAF0803193B2C2F08840083132030F6
:100870008000AF0A412C20300A128A1525240A1262
:100880008A11AC032C08803A7E3E0318302C0230CB
:10089000AA072A02840083130008AE00252D023027
:1008A000AA072A02840083130008B200840A000801
:1008B000B300AE012E083207C7003308C80047084E
:1008C0000318C80A0A128A111B200A128A1100385A
:1008D00003196C2CAE0A5A2C2B082E020318722C0A
:1008E0002E08AB002B08AC1BA92CFF3A2C07031CCD
:1008F000A92CAD0AAF080319842C2F088400831398
:1009000020308000AF0A8A2C20300A128A15252454
:100910000A128A11AC03722C3308C80032080A127A
:100920008A111B200A128A11AE00B20A0319B30AF7
:10093000AD0AAF080319A32C2F08840083132E08D7
:100940008000AF0AA92C2E080A128A1525240A1243
:100950008A11AB032B0F8C2C342D2808C8002708D4
:100960000A128A111B200A128A112A3A031DBF2C6F
:100970000230AA072A02840083130008E32C280807
:10098000C80027080A128A111B20D03EAB00A70A14
:100990000319A80A2808C80027080A128A111B2070
:1009A0000A128A11AE0030302E02031CE72C3A30B6
:1009B0002E020318E72C0A30F1002B080A128A15C0
:1009C00032242E07D03EAB00A70A0319A80A280834
:1009D000C8002708A70A0319A80A0A128A111B20AF
:1009E0000A128A11AE00003A0319502B2A3A031951
:1009F000592B043A0319AD2C763A0319622B3B3A72
:100A00000319422C073A0319602B0B3A0319642B84
:100A10001C3A03194F2C063A0319662B0D3A031999
:100A2000622B30302E02031C252D3A302E02031883
:100A3000252D0A30F1002C080A128A1532240A12D8
:100A40008A112E07D03EAC00E72CAD0AAF0803197F
:100A5000302D2F08840083132E088000AF0A342D18
:100A60002E080A128A1525242808C8002708A70A74
:100A70000319A80A0A128A111B200A128A11AE0051
:100A8000AE08031D472BAF0803194A2D2F08840019
:100A9000831380012D080800293083120313BA0044
:100AA000C1012608BC00A12F831203133B08253A7D
:100AB00003195B2D5C2D642DC10A3B080A128A15AF
:100AC000CD240A128A11A12FFF3083120313BE0016
:100AD000C201BD01742F83120313BA080319712DCB
:100AE000722D762D3A08840083138001831203133C
:100AF0004108C32F023083120313BC073C02840059
:100B000083130008C2006A2D83120313BD0A902DBF
:100B1000083083120313BE07FE3083120313BE078F
:100B2000023083120313BC073C02840083130008C5
:100B3000BF00840A0008C0003D1C9F2DA02DAF2DD2
:100B4000C01FA32DA42DAB2DBF09C009BF0A0319D7
:100B5000C00AC203AE2D83120313BD01B22D83124E
:100B60000313BD010B3083120313BE07831203135B
:100B70003E08F200F3014008F1003F08F0000A12BD
:100B80008A11C6270A128A117008BB003E08F200BB
:100B9000F3013F08F0004008F1000A128A11C6274D
:100BA0000A128A117408BF007508C000C301C30A85
:100BB000C401ED2D831203133E08F200F301430834
:100BC000F0004408F1000A128A155E240A128A1104
:100BD0007408C3007508C400C203831203134408D9
:100BE0004002031DF52D43083F020318F82DF92D8F
:100BF000DA2D032E83120313C10A20300A128A153C
:100C0000CD240A128A1183120313C2034208803AC8
:100C10007F3E03180C2E0D2EFA2D831203133D1C5C
:100C2000122E132E1A2EC10A2D300A128A15CD2427
:100C30000A128A114B2E831203134408F30043084F
:100C4000F2004008F1003F08F0000A128A11C6279E
:100C50000A128A117408F0007508F1003E08F200CB
:100C6000F3010A128A11C6270A128A117008C200FB
:100C70004208803A763E031C3E2E3F2E412E07301E
:100C8000C20783120313C10A4208303E0A128A15B2
:100C9000CD240A128A11831203133E08F200F301D5
:100CA0004308F0004408F1000A128A11C6270A120C
:100CB0008A117408C3007508C40044084304031D66
:100CC000622E632E1B2E0A30831203133B02031C79
:100CD0006A2E6B2E6D2E0730BB0783120313C10AD9
:100CE0003B08303E0A128A15CD240A128A11A12F20
:100CF000832E83120313C10A20300A128A15CD24D1
:100D00000A128A11C203831203134208803A7E3EFC
:100D100003188B2E8C2E792E023083120313BC07FE
:100D20003C02840083130008BB00C10A3B080A127E
:100D30008A15CD240A128A11A12F023083120313BF
:100D4000BC073C02840083130008C300840A000827
:100D5000C400BB01AE2E83120313BB0A831203131C
:100D60003B084307C7004408C80047080318C80ADF
:100D70000A128A111B200A128A110038031DC12E83
:100D8000C22EAB2E831203133E083B020318C92E5A
:100D9000CA2ECC2E3B08BE00D72E83120313C10AE5
:100DA00020300A128A15CD240A128A11C203831236
:100DB00003133E08C21BE22EFF3A42070318E12E3E
:100DC000E22ECD2EF82E831203134408C8004308E8
:100DD0000A128A111B200A128A11BB00C30A0319C6
:100DE000C40AC10A3B080A128A15CD240A128A11C4
:100DF00083120313BE033E0FFE2EFF2EE32EA12F00
:100E0000831203132808C80027080A128A111B201E
:100E10000A128A112A3A031D0E2F0F2F1A2F0230A1
:100E2000BC073C02840083130008BE00A70A031914
:100E3000A80A4D2F831203132808C80027080A1296
:100E40008A111B200A128A11D03EBE00A70A03197C
:100E5000A80A2808C80027080A128A111B200A12AB
:100E60008A11BB0030303B02031C3D2F372F3A3034
:100E70003B0203183D2F3C2F3F2F3E2F4D2F0A30B2
:100E8000F1003E080A128A1532240A128A113B0721
:100E9000D03EBE00A70A0319A80A6A2D303083127B
:100EA00003133B02031C5B2F552F3A303B02031800
:100EB0005B2F5A2F5D2F5C2F692F0A30F1004208FB
:100EC0000A128A1532240A128A113B07D03EC20048
:100ED0006A2D83120313C10A3B080A128A15CD2416
:100EE0000A128A11A12FA12F831203132808C80008
:100EF0002708A70A0319A80A0A128A111B200A1236
:100F00008A11BB00003A03196B2D2A3A03197A2D76
:100F1000043A0319002F763A0319882D3B3A031936
:100F2000782E073A0319842D0B3A03198C2D1C3A9D
:100F300003199D2E063A0319902D0D3A0319882D99
:100F40004E2F831203132808C8002708A70A031985
:100F5000A80A0A128A111B200A128A11BB00BB08B8
:100F6000031DB32FB42F542D83120313BA08031992
:100F7000BA2FBB2FBF2F3A0884008313800183123E
:100F800003134108C32F031383120800F601F40171
:100F9000F50172087304031DD02FF001F101003434
:100FA0001F30F6040310F60AF20DF30D031CD32FC5
:100FB000F30CF20C73087102031DE02F720870022B
:100FC000031CE82F7208F0027308031C730AF10275
:100FD000F40DF50DF60BF61AD82FF61FF42FF409C1
:100FE000F40A0319F503F5097408F2007508F30013
:100FF000761F0034F009F00A0319F103F1090034F7
:10184A00830108000E30831603139F004130831270
:10185A009F000C13031383120800F0000030711864
:10186A0070070310F00D0310F10CF10803190800BA
:10187A00342C831203138511A6002608803E0A120F
:10188A008A1589240A128A150313831208008312FF
:10189A000313851101300A128A1589240A128A153E
:1018AA0002300A128A15AB240A128A15031383120C
:1018BA000800F401F5010310F30CF20C031C6C2C64
:1018CA007008F40771080318710AF5070310F00D80
:1018DA00F10D7208730403190034602C8316031384
:1018EA008611831286118316871507168030940095
:1018FA002830831294000930831693008312130848
:10190A00A60003138312080083120313A700270EED
:10191A000F39F0000808F039700488008514851022
:10192A0027080F39F0000808F03970048800851478
:10193A0085100D30A800A22CA22C83120313A80B29
:10194A00A72CA82CA12C03138312080083120313BB
:10195A00A800043083120313A70053308312031321
:10196A00A900B82CB82C83120313A90BBD2CBE2CCA
:10197A00B72C83120313A70BC32CC42CB22C8312CB
:10198A000313A80BC92CCA2CAE2C0313831208000C
:10199A00831203138515C500450E0F39F000080898
:1019AA00F039700488008514851045080F39F00055
:1019BA000808F03970048800851485100D30C600B7
:1019CA00E72CE72C83120313C60BEC2CED2CE62C28
:1019DA00031383120800F0308316031388050E30B0
:1019EA009F00F13085058312051185110F300A1207
:1019FA008A15AB240A128A150330880085148510CB
:101A0A0005300A128A15AB240A128A158514851024
:101A1A002130A600112D112D83120313A60B162DAA
:101A2A00172D102D831203138514851005300A1201
:101A3A008A15AB240A128A1502308800851485108B
:101A4A000D30A600292D292D83120313A60B2E2D46
:101A5A002F2D282D28300A128A1589240A128A1550
:101A6A0008300A128A1589240A128A150F300A12B6
:101A7A008A1589240A128A1506300A128A158924B7
:101A8A000A128A150313831208008316031311140A
:101A9A004E2D831603131118532D542D4E2D8312D8
:101AAA0003138C119A3093005A2D831203138C1D41
:101ABA005F2D602D5A2D831203138C119301652D0E
:101ACA00831203138C1D6A2D6B2D652D8316031348
:101ADA0091146F2D831603139118742D752D6F2D84
:101AEA00831203138C119B3093007B2D83120313F3
:101AFA008C1D802D812D7B2D831203138C1183164F
:101B0A009115872D83160313141C8C2D8D2D872D6B
:101B1A00831203131308A60083161116942D831635
:101B2A000313111A992D9A2D942D83160313111547
:101B3A009E2D831603131119A32DA42D9E2D8312F6
:101B4A0003132608A82D0313831208008316031310
:101B5A001114AF2D831603131118B42DB52DAF2D03
:101B6A00831603139112111783128C11C430930038
:101B7A00BE2D831203138C1DC32DC42DBE2D8312BB
:101B8A0003138C118316111BCB2DCE2D83128615B0
:101B9A00D02D8312861183160313111783128C1109
:101BAA009301D72D831203138C1DDC2DDD2DD72D28
:101BBA00831203138C118316111BE42DE72D831254
:101BCA008615E92D831286118316031311178312C2
:101BDA008C1101309300F12D831203138C1DF62D05
:101BEA00F72DF12D831203138C118316111BFE2D71
:061BFA00012E8312861586
:101C0000032E831286118316031311171115082E44
:101C10008316031311190D2E0E2E082E0313831293
:101C20000800831603131114152E831603131118BD
:101C30001A2E1B2E152E83160313911211178312C1
:101C40008C11C4309300242E831203138C1D292E73
:101C50002A2E242E831203138C118316111B312E6E
:101C6000342E83128615362E8312861183160313A3
:101C7000111783128C11013093003E2E831203132F
:101C80008C1D432E442E3E2E831203138C1183167B
:101C9000111B4B2E4E2E83128615502E8312861149
:101CA0008316031311171115552E831603131119DB
:101CB0005A2E5B2E552E8316031311145F2E831696
:101CC00003131118642E652E5F2E831603139112D1
:101CD00083128C11C53093006D2E831203138C1D5B
:101CE000722E732E6D2E831203138C118316911591
:101CF000792E83160313141C7E2E7F2E792E8312C9
:101D000003131308A20083161116862E83160313DD
:101D1000111A8B2E8C2E862E831603131115902EDE
:101D2000831603131119952E962E902E83120313EA
:101D3000861522089B2E03138312080083160313B3
:101D40001114A22E831603131118A72EA82EA22E4B
:101D5000831603139112111783128C11C430930050
:101D6000B12E831203138C1DB62EB72EB12E831203
:101D700003138C118316111BBE2EC12E83128615E0
:101D8000C32E8312861183160313111783128C112D
:101D90009301CA2E831203138C1DCF2ED02ECA2E70
:101DA000831203138C118316111BD72EDA2E831284
:101DB0008615DC2E831286118316031311178312E6
:101DC0008C119301E32E831203138C1DE82EE92E50
:101DD000E32E831203138C118316111BF02EF32EA6
:101DE00083128615F52E831286118316031311179D
:101DF00083128C119301FC2E831203138C1D012F6F
:101E0000022FFC2E831203138C118316111B092F32
:101E10000C2F831286150E2F83128611831603133F
:101E2000111783128C1105309300162F83120313A0
:101E30008C1D1B2F1C2F162F831203138C1183163E
:101E4000111B232F262F83128615282F831286110C
:101E500083160313111783128C1103309300302F54
:101E6000831203138C1D352F362F302F831203134B
:101E70008C118316111B3D2F402F83128615422F84
:101E80008312861183160313111783128C114F309E
:101E900093004A2F831203138C1D4F2F502F4A2F6C
:101EA000831203138C118316111B572F5A2F831281
:101EB00086155C2F83128611831603131117831264
:101EC0008C114B309300642F831203138C1D692FE8
:101ED0006A2F642F831203138C118316111B712F29
:101EE000742F83128615762F83128611831603139F
:101EF000111783128C1193017D2F831203138C1DF4
:101F0000822F832F7D2F831203138C118316111BB5
:101F10008A2F8D2F831286158F2F83128611831699
:101F2000031311171115942F831603131119992FE9
:101F30009A2F942F8316031311149E2F83160313C5
:101F40001118A32FA42F9E2F83160313911211177C
:101F500083128C11C4309300AD2F831203138C1D98
:101F6000B22FB32FAD2F831203138C118316111BC5
:101F7000BA2FBD2F83128615BF2F831286118316A9
:101F80000313111783128C119301C62F83120313AD
:101F90008C1DCB2FCC2FC62F831203138C118316CD
:101FA000111BD32FD62F83128615D82F831286119B
:101FB00083160313111783128C1140309300E02F06
:101FC000831203138C1DE52FE62FE02F83120313DA
:101FD0008C118316111BED2FF02F83128615F22F13
:101FE000831286118316031311171115F72F831609
:101FF00003131119FC2FFD2FF72F03138312080071
:02400E00393542
:00000001FF
